:100000000C9466000C9487000C9487000C94870075
:100010000C9487000C9487000C9487000C94870044
:100020000C9487000C9487000C9487000C94870034
:100030000C9487000C9487000C9487000C94870024
:100040000C9487000C9487000C9487000C94870014
:100050000C9487000C941C030C9487000C9487006C
:100060000C9487000C94D8070C9487000C9487009C
:100070000C9487000C9487000C9487000C948700E4
:100080000C9487000C9487000C9487000C947E07D6
:100090000C94920E0C9487000C9487000C948700AB
:1000A0000C9487000C9487000C9487000C948700B4
:1000B0000C9487000C9487000C9487000C948700A4
:1000C0000C9487000C9487000C94870011241FBEA9
:1000D000CFEFD1E2DEBFCDBF00E00CBF13E0A0E068
:1000E000B2E0EEEEF9E300E00BBF02C007900D9224
:1000F000A436B107D9F714E0A4E6B3E001C01D921D
:10010000AB3EB107E1F70E949A020C94F51C0C94E7
:100110000000EEE6F0E080818260808383E084BDB1
:1001200085BD8AEF87BD0895E1E7F0E080818160B9
:100130008083089580917100817008958091960365
:10014000982F9295969596959370282F221F222787
:10015000221F9227282F22952F709227282F26952D
:10016000269592279170880F892B80939603089586
:10017000FC0107C08091C80085FFFCCF9093CE00A2
:10018000319690819923B1F708951F93CF93DF9310
:10019000182F492FE0E1F7E2C0E0D0E0812F942F43
:1001A000BF010E94BF1C9B016115710549F0809140
:1001B000C80085FFFCCF822F805D8093CE001EC0DB
:1001C000812F942FBF010E94BF1C182F492FCF01F0
:1001D0006AE070E00E94BF1CFB012196C430D1058B
:1001E000E9F619C08091C80085FFFCCF812F942FBC
:1001F000BF010E94BF1C605D6093CE00812F942FD1
:10020000BF010E94BF1C182F492FCF016AE070E088
:100210000E94BF1CFB01309729F7DF91CF911F91FE
:100220000895982F9F709A3030F48091C80085FF10
:10023000FCCF905D05C08091C80085FFFCCF995C24
:100240009093CE000895CF93DF93EC01892F9927E7
:1002500082958F70009711F00E9411018D2F9927C0
:10026000009711F00E941101CE0124E09695879528
:100270002A95E1F7009711F00E9411018C2F0E943E
:100280001101DF91CF910895982F8091C80085FFCB
:10029000FCCF9093CE0080E090E008952091C800BC
:1002A000332727FD30952227330F221F3327C9011B
:1002B00008958091C80087FFFCCF8091CE0090E028
:1002C0000895F999FECF92BD81BDF89A80B5089541
:1002D000F999FECF92BD81BD60BDF894FA9AF99A62
:1002E000789408958091C90088618093C90083E360
:1002F0008093CC001092CD0009C08091C80087FF88
:10030000FCCF8091CE008AE00E94AE078091C800A9
:1003100087FDF3CF8091C90080688093C9008091E8
:10032000C10088698093C1008FE18093C40010925E
:10033000C50090EC91B98CE382B987E384B995B993
:100340009FEF97B988EF8AB98BE08BB982E08DB9BE
:100350009EB910BA91BB13BA94BB81E58CBD0895C8
:10036000EF92FF920F931F938C0181E00D321807DB
:1003700018F00CE211E005C00431110510F404E19D
:1003800010E010939303009392031093950300934E
:10039000940385E090E0612F0E94680186E090E080
:1003A000609192030E94680180919203909193035F
:1003B0000E94520E980140E050E060E070E788E350
:1003C00099E30E94D31CB901CA0123E09695879551
:1003D000779567952A95D1F726E030E040E050E028
:1003E0000E94D31C79018A01C801AA27BB279C015E
:1003F000887F892B69F4B3E016950795F794E79405
:10040000BA95D1F7F0929803E092970382E051C039
:10041000C901807F892B69F4A4E016950795F794AC
:10042000E794AA95D1F7F0929803E092970386E0BB
:1004300040C0C901807E892B69F4F5E016950795C7
:10044000F794E794FA95D1F7F0929803E092970326
:1004500087E02FC0C901807C892B69F4E6E01695FE
:100460000795F794E794EA95D1F7F0929803E09214
:10047000970383E01EC0C9018070892B51F4BB270C
:10048000A12F902F8F2D909398038093970384E052
:1004900010C020703C7F232B79F46AE016950795F5
:1004A000F794E7946A95D1F7F0929803E092970356
:1004B00085E08093910002C0109291008091970393
:1004C00090919803909581959F4F90939803809376
:1004D000970390939500809394001F910F91FF9044
:1004E000EF900895F999FECF85E090E092BD81BD2F
:1004F000F89A30B5F999FECF86E090E092BD81BDC3
:10050000F89A20B5932F80E030E0822B932B0E9445
:10051000B001109265038091710081608093710039
:10052000089585E20E940D0CE1E7F0E080818E7F66
:10053000808308950F931F930E9472010E9472029C
:1005400080916E00826080936E0083E084BD85BDE3
:100550008AEF87BD80919203809396030E94D80909
:100560000E94A309789412E001E00E94E50A8091BC
:10057000C103883009F444C0893088F4833019F10C
:10058000843030F4813039F1823008F050C02EC010
:100590008530E1F0853078F1873039F717C08C303D
:1005A00009F440C08D3018F48A30E9F440C08E3030
:1005B00029F08E30A8F08F30C1F612C0109264037B
:1005C0000E942B0ED2CF109264032EC000936403BE
:1005D0000E944219CACF109264030E943812C5CFFC
:1005E00010926403F5CF10936403F2CF109264036A
:1005F0000E942109BACF109264030E94DF0FB5CF89
:1006000010926403809171008160809371000E9458
:10061000380C0E94E50A8091C1038830D1F30E9412
:100620009102A3CF109364030E9406169ECF0E94EE
:10063000380C0E94600D99CF1F920F920FB60F9247
:100640000BB60F9211241F932F933F934F935F93F9
:100650006F937F938F939F93AF93BF93EF93FF938A
:1006600030B1327090B180919903381799F1292FE8
:100670002170332339F080919403909195032223C4
:1006800039F008C08091940390919503222311F0D2
:10069000019601C0019790939503809394038091F4
:1006A0009403909195038D52914030F08CE291E04B
:1006B0009093950380939403809194039091950374
:1006C000449730F484E190E09093950380939403F1
:1006D00030939903809176038F3F29F080917603C0
:1006E0008F5F8093760380918E0390918F038F5F4D
:1006F0009F4F49F080918E0390918F0301969093C4
:100700008F0380938E0380918303909184038F5F86
:100710009F4F49F0809183039091840301969093B9
:10072000840380938303109164031130B9F08091A6
:10073000700390917103892B59F18091700390910E
:1007400071030197909371038093700380917003FC
:1007500090917103892BE1F45C981AC099B192953C
:10076000917080917403882389F4992379F08091A2
:100770006E0390916F03019690936F0380936E03C5
:1007800088EF0E9486081093740302C0909374034C
:100790008091710080FD14C080916703883C29F42A
:1007A000109267030E947E0D06C080916703843615
:1007B00011F40E94710D809167038F5F809367032E
:1007C000FF91EF91BF91AF919F918F917F916F9129
:1007D0005F914F913F912F911F910F900BBE0F9002
:1007E0000FBE0F901F9018950F931F93F894809150
:1007F00064038150823020F18091C103843001F183
:1008000080916D03863010F010926D0380916D031E
:1008100080FF02C05C9804C05C9A88EF0E94860842
:1008200080916D03882339F080916D038F5F8093F1
:100830006D03789460C380916D038F5F80936D0327
:1008400080916503883010F01092650380916503F4
:1008500080FFFBC18091C103883029F1893080F489
:10086000833009F486C0843020F4813009F028C335
:1008700022C0853009F43BC1873009F021C39CC0F8
:100880008C3009F476C08D3038F4893009F42FC1EA
:100890008B3009F015C390C08D3009F428C18F301A
:1008A00009F00EC389C080E00E94D80F80919103A7
:1008B0000E945E0805C380917704882321F480910B
:1008C0006C04882361F0909191039F3F41F08091E7
:1008D0008A03991F9927991F892B0E94D80F80910D
:1008E0006C04882309F4ECC280917404803148F4CC
:1008F000E0917404F0E0E758FB4F80818F3F09F0EE
:10090000DFC210927404809173048F5F809373042C
:1009100080917304803160F4E0917304F0E0EE0F95
:10092000FF1FE45BFB4F808191818F5F9F4F11F42C
:1009300010927304E0917304F0E0EE0FFF1FE45B8C
:10094000FB4F8081918190936F0480936E0480911E
:100950006E0490916F048F5F9F4F21F48FEF80930F
:100960007904AEC20E949711809385030E944D0CBA
:10097000A7C280917704882309F4A2C280919103D1
:100980008F3F29F0881F8827881F0E94D80F8091E9
:1009900074048F5F8093740480917404803148F4F0
:1009A000E0917404F0E0E758FB4F80818F3F09F03D
:1009B00087C21092740484C28091CA04882309F407
:1009C0007FC2909191039F3FE9F080918A03991F24
:1009D0009927991F982B21F081E00E94D80F12C00F
:1009E00080E00E94D80F20919103822F90E08F73B6
:1009F0009070892B21F080918503820F01C0822F96
:100A00000E945E08209166032F3FA9F090918A030F
:100A1000822F881F8827881F892B69F0822F90E0FA
:100A20008F739070892B21F080918503820F01C014
:100A3000822F0E945E0880917404803148F4E09116
:100A40007404F0E0E758FB4F80818F3F09F038C213
:100A5000109274048091C9048F5F8093C9048091BF
:100A6000C904803240F4E091C904F0E0E755FB4F3F
:100A700080818F3F11F41092C90489E894E069EAFB
:100A800074E00E942919882331F090918C038091A1
:100A90008D039817C9F020E030E0F901E757FB4FCC
:100AA0008081F901E755FB4F80832F5F3F4F203254
:100AB000310599F71092C9041092850310928603AC
:100AC0000E94400D0E948C0D80918D0380938C03B9
:100AD000809186038093850380918C03E091C90403
:100AE000F0E0E755FB4F60810E94D415E9C1809189
:100AF000CA04882309F4E4C1909191039F3F21F136
:100B000080918A03991F9927991F982B21F081E0E2
:100B10000E94D80F19C080E00E94D80F0091910365
:100B2000802F90E08F739070892B59F0109185037E
:100B300080916E0490916F040E94FE10100F810F3F
:100B400001C0802F0E945E0880917404803148F4B7
:100B5000E0917404F0E0E758FB4F80818F3F09F08B
:100B6000AFC110927404809173048F5F80937304FB
:100B700080917304803168F4E0917304F0E0EE0F2B
:100B8000FF1FE45BFB4F808191818F5F9F4F09F0D6
:100B90004CC0109273048091C9048F5F8093C90484
:100BA0008091C904803240F4E091C904F0E0E75537
:100BB000FB4F80818F3F79F51092C90489E894E05A
:100BC00069EA74E00E942919882331F090918C031E
:100BD00080918D039817B9F020E030E0F901E757D4
:100BE000FB4F8081F901E755FB4F80832F5F3F4F1B
:100BF0002032310599F710928503109286030E94E6
:100C0000400D0E948C0D80918D0380938C03809108
:100C100086038093850380918C03E091C904F0E002
:100C2000E755FB4F60810E943D11E0917304F0E0B5
:100C3000EE0FFF1FE45BFB4F8081918190936F0467
:100C400080936E040E9497113BC18091C10388304C
:100C500029F1893080F4833009F493C0843020F482
:100C6000813009F02DC12CC0853009F4C0C0873017
:100C700009F026C1B2C08C3009F483C08D3038F43D
:100C8000893009F4B4C08B3009F01AC1A6C08D3088
:100C900009F4ADC08F3009F013C19FC0809191035A
:100CA0008093660380919003809391030E949E003D
:100CB00080939003809191038F7360E040E0FAC0CD
:100CC00080917704882329F480916C04882309F4A7
:100CD000F7C080917704882371F08091740480318B
:100CE00040F4E0917404F0E0E758FB4F80818F3FBF
:100CF00011F41092740480919103809366038091A3
:100D00007404E82FF0E0E758FB4FE081E093910393
:100D10008F5F80937404EF3F09F4D2C080918B03FE
:100D2000882319F0E07CE093910320919103822FB6
:100D300090E08F73907060916603322F3F73422F63
:100D40004295469546954370892B79F080918A03A8
:100D50009091890320918503661F6627661F682B83
:100D60004170492B832F820F35C080918A03909167
:100D70008903661F6627661F682B4170492B832FE6
:100D800029C080917704882309F49AC00E944D0CF1
:100D9000809174040E945B0C8091910380936603A0
:100DA000E0917404F0E0E758FB4F80818093910359
:100DB0008F3F09F485C00E94BB0D80919103609123
:100DC0006603661F6627661F482F4295469546951F
:100DD00041708F730E94C20F73C08091CA04882330
:100DE00031F00E944D0C809174040E945B0C809144
:100DF000CA04882309F464C0809191038093660338
:100E000080917404E82FF0E0E758FB4FE081E09315
:100E100091038F5F80937404EF3F09F451C0809178
:100E20008B03882319F0E07CE093910340919103B8
:100E3000842F90E08F739070042F0F73892B51F1E2
:100E40001091850380916E0490916F040E94FE10B2
:100E500090918A0320918903100F60916603661FA9
:100E60006627661F692B40919103429546954695EA
:100E70004170422B810F0E94C20F0091910310918B
:100E8000850380916E0490916F040E94FE10100FF4
:100E9000810F14C080918A03909189036091660349
:100EA000661F6627661F682B4295469546954170DA
:100EB000492B802F0E94C20F809191030E94270826
:100EC00080916503843030F485E20E94B20B0E9469
:100ED0007E0D09C080916503883028F485E20E9468
:100EE0000D0C0E94710D0E94600D809165038F5F53
:100EF0008093650378941F910F9108951F920F922C
:100F00000FB60F920BB60F9211242F933F934F936E
:100F10005F936F937F938F939F93AF93BF93EF9361
:100F2000FF938091970390919803909395008093FD
:100F300094000E94F403FF91EF91BF91AF919F91B4
:100F40008F917F916F915F914F913F912F910F9072
:100F50000BBE0F900FBE0F901F90189520EA3FE038
:100F6000E22FF32F3197F1F78A95D1F708959AEF91
:100F700020EA3FE019C0E22FF32F3197F1F79A955D
:100F8000D1F7E22FF32F3197F1F79A95D1F7E22FAE
:100F9000F32F3197F1F79A95D1F7E22FF32F31978D
:100FA000F1F79A95D1F78150882309F0E4CF08959D
:100FB0001F920F920FB60F920BB60F9211248F93C0
:100FC0009F93EF93FF939091C600983FB1F4809167
:100FD0006403813021F05C9A85E0809370038091F6
:100FE000CA04882349F18091690390916A030196AC
:100FF00090936A03809369031FC080916C03E82F6C
:10100000F0E0E556FC4F90838F5F80936C038091F6
:101010006C038F7180936C0390916C0380916B03D0
:10102000981751F480916B038F5F80936B038091CD
:101030006B038F7180936B03FF91EF919F918F9161
:101040000F900BBE0F900FBE0F901F901895282F7A
:1010500090919A038091C00085FFFCCF9069909396
:10106000C600822F90E08F739070892B39F48091A5
:10107000C00085FFFCCF1092C60009C08091C0005F
:1010800085FFFCCF822F8F73875E8093C600822FEF
:10109000829586958695837080FF07C090910002A7
:1010A0008091C00085FFFCCF06C090910202809124
:1010B000C00085FFFCCF9093C6000895282F909123
:1010C0009A038091C00085FFFCCF90689093C60082
:1010D000822F90E08F739070892B39F48091C0003B
:1010E00085FFFCCF1092C60008C08091C00085FF2C
:1010F000FCCF2F73275E2093C60090910102809150
:10110000C00085FFFCCF9093C6000895982F809172
:10111000C00085FFFCCF9093C60080E090E008956A
:1011200090916B0380916C0320E030E0981711F0F0
:1011300021E030E0C901089590916B0380916C0328
:101140009817D1F3F89490916B03E92FF0E0E556EE
:10115000FC4F80819F5F90936B0390916B039F7115
:1011600090936B03789490E0089590916B03809135
:101170006C039817B9F00E949C08482F87FF12C093
:10118000582F52955F705F3071F0282F30E02F702C
:1011900030708091BB0390E02817390719F4509301
:1011A000680301C040E0842F089590919A038091D4
:1011B000C00085FFFCCF906B9093C6008091C0006B
:1011C00085FFFCCF8BE78093C6008091C00085FF30
:1011D000FCCF1092C600089580916403823049F0DC
:1011E0008091C00085FFFCCF8CEF8093C6000E94E9
:1011F000D508089590916603891731F480E00E9424
:10120000D80F8FEF8093660308951F93182F962FA2
:10121000662321F460E00E94FA0811C060E080912A
:1012200066038F3F09F061E0812F8951953610F0F8
:1012300041E001C040E00E94C20F109366031F917D
:1012400008950F931F930E9491020E944D0C80916C
:10125000BB030E945B0C0E94E50A84E60E94AE0775
:101260000E94E50A84E60E94AE070E94E50A00910A
:10127000C8038FEF809366030E94E50A8091C10343
:10128000882329F00E94D5081F910F91089560913D
:10129000C803061771F06093BB0383E090E00E94DF
:1012A00068010E944D0C8091BB030E945B0C009171
:1012B000C80390916B0380916C039817E9F20E9428
:1012C0009C08482F87FF15C0582F52955F705F30DC
:1012D00051F0282F30E02F7030708091BB0390E0E8
:1012E0002817390719F45093680303C01092680354
:1012F000C3CF80916803883089F0893009F0BCCF72
:1013000047FD02C0142F03C00E949C08182F0E94A2
:101310009C08682F812F0E940509AECF47FD02C0AF
:10132000142F03C00E949C08182F0E949C08682F4D
:10133000812F0E94FA08A0CF90E00E9461018031C5
:1013400008F08FE0089583E00E949C098093BB031E
:1013500084E00E949C0980939A030895809164031D
:10136000813009F05F98089599B1991F9927991FC5
:1013700080917203882331F4992321F090937203B2
:1013800081E008959093720380E0089599B1991FC8
:101390009927991F80917303882331F0992321F4B1
:1013A0001092730381E008959093730380E0089591
:1013B0008AB1806F8AB98BB18F708BB908958AB169
:1013C0008F708AB98BB18F708BB908951F930E946B
:1013D0009A00182F809164038130D1F0112311F00D
:1013E0000E9491025C985F9A85E00E94AE0780910E
:1013F0009703909198030A97909395008093940097
:1014000010926D0310926503112311F00E94940055
:101410001F910895AC01F894289800000000000086
:101420000000289A20E030E01EBC0DB407FEFDCF7E
:101430008EB5FA01E20FF31F80832F5F3F4F2330F9
:10144000310591F77894089516980895169A08959D
:1014500020B1269526952F70822F90E02695322F69
:10146000369536952270322B880F991F282F2470BD
:10147000322B880F991F880F991F8870382B8FE0A7
:10148000831B089580B1869586958F700895282FC7
:10149000883110F080E00895E82FE695E695E6950E
:1014A000F0E0EE53FC4F808190E0277002C09595EC
:1014B00087952A95E2F781700895282F883110F0DA
:1014C00080E00895E82FE695E695E695F0E0E25491
:1014D000FC4F808190E0277002C0959587952A95F2
:1014E000E2F781700895282F883110F080E0089588
:1014F000E82FE695E695E695F0E0EB53FC4F80810A
:1015000090E0277002C0959587952A95E2F7817043
:1015100008958091C203882359F48091C3038823DE
:1015200039F490E08091C403882319F491E001C05C
:1015300090E0892F08951F93CF93DF93CBE0D2E003
:1015400010E088810E94470A882329F41F5F2196B2
:101550001D30B9F71FEF812FDF91CF911F910895B3
:101560001F93CF93DF93C3E0D2E010E088810E9405
:10157000470A912F9F5F882311F0892F05C0192FEB
:101580002196983099F780E0DF91CF911F910895CF
:101590001F93CF93DF93C3E0D2E010E088810E94D5
:1015A0005D0A912F9F5F882311F0892F05C0192FA5
:1015B0002196983099F780E0DF91CF911F9108959F
:1015C00080917503109275030895EF92FF920F9327
:1015D0001F93DF93CF9300D000D0CDB7DEB720911B
:1015E000940330919503809192039091930328176F
:1015F000390731F080919403909195030E94B001D6
:101600001092BE031092C5031092BF031092C6033E
:101610001092C0031092C70380917603843108F4BE
:1016200094C01092760316988E010F5F1F4FC80169
:101630000E940A0A8091C2038C838091C3038D8328
:101640008091C4038E8340E050E061E0E62EF12CEF
:10165000E42FE695E695E695F0E0BF016E537C4FEA
:10166000DB013C91CA0187709070D70102C0AA0FBC
:10167000BB1F8A95E2F7CD01DF01A753BC4FAC91A8
:10168000A823E00FF11FE081E823232F2823809572
:10169000222311F0EA2B01C0EA238323E82BDB018C
:1016A000EC934F5F5F4F4831510591F60E94280A35
:1016B000982F8091C803981749F08091BD0398171F
:1016C00029F49093C80381E0809375039093BD0340
:1016D000169A40E050E08E010F5F1F4FBE016C5F15
:1016E0007F4FDA01A753BC4FF801E40FF51F80814B
:1016F0008C93FB01E40FF51F2081FA01EE53FC4FA0
:101700009081FA01E254FC4F822F809589238083D7
:10171000FA01EB53FC4F9095922390834F5F5F4FFC
:1017200043305105F1F690B1969596959F70809152
:10173000C103981731F08091BC03981711F490936E
:10174000C1039093BC030E94600D26960FB6F894D7
:10175000DEBF0FBECDBFCF91DF911F910F91FF90E4
:10176000EF900895282F883290F4E82FE695E695BB
:10177000E695F0E0E958FC4F277081E090E002C068
:10178000880F991F2A95E2F72081282B208308953E
:10179000282F883290F4E82FE695E695E695F0E05C
:1017A000E458FC4F277081E090E002C0880F991F39
:1017B0002A95E2F72081282B20830895282F88324C
:1017C00098F4E82FE695E695E695F0E0E458FC4FAE
:1017D000277081E090E002C0880F991F2A95E2F7F8
:1017E00080952081822380830895E82F883210F02D
:1017F00020E011C0282F277081E090E002C0880F00
:10180000991F2A95E2F7E695E695E695F0E0E4580B
:10181000FC4F20812823822F0895282F883298F4A6
:10182000E82FE695E695E695F0E0E958FC4F27703D
:1018300081E090E002C0880F991F2A95E2F7809519
:101840002081822380830895982F9695969596956A
:10185000E7E7F3E0E90FF11D208130E0877002C077
:10186000359527958A95E2F721703070C901089562
:1018700010927B0310927A031092790310927803EE
:10188000109277031092800310927F0310927E03D0
:1018900010927D0310927C030895CF93DF93C5E4EB
:1018A000D2E089910E940D0C82E0C535D807C9F7B6
:1018B000DF91CF910895803138F4E82FF0E0EB5BB1
:1018C000FD4F80810E94B20B0895803138F4E82FDB
:1018D000F0E0EB5BFD4F80810E94C80B08958031E2
:1018E00010F080E00895E82FF0E0EB5BFD4F808181
:1018F0000E94240C0895803110F080E00895E82FB4
:10190000F0E0EB5BFD4F80810E94F50B089588317C
:1019100038F4E82FF0E0E35DFD4F80810E94B20BC8
:101920000895883138F4E82FF0E0E35DFD4F8081C1
:101930000E94C80B0895883138F4E82FF0E0E35D89
:10194000FD4F80810E940D0C0895CF93DF93CDE26F
:10195000D2E089910E940D0C82E0C534D807C9F706
:10196000DF91CF910895E82F8150883030F4F0E076
:10197000EC5DFD4F80810E94B20B08950F931F9381
:10198000CF93DF93082FC5E2D2E011E0101741F4A6
:10199000E12FF0E0EC5DFD4F80810E94B20B03C0AF
:1019A00088810E940D0C1F5F2196193079F7DF9115
:1019B000CF911F910F910895E82F8150883030F416
:1019C000F0E0EC5DFD4F80810E940D0C0895E82F42
:1019D0008150883030F4F0E0EC5DFD4F80810E9452
:1019E000C80B0895E82F8150883010F080E00895EA
:1019F000F0E0EC5DFD4F80810E94F50B0895E82F2B
:101A00008150883010F080E00895F0E0EC5DFD4FEB
:101A100080810E94240C0895CF93DF93C5E2D2E029
:101A200089910E940D0C82E0CD32D807C9F7DF9171
:101A3000CF9108958D3038F4E82FF0E0E85EFD4F47
:101A400080810E94B20B08958D3038F4E82FF0E0C9
:101A5000E85EFD4F80810E940D0C08958D3038F4B2
:101A6000E82FF0E0E85EFD4F80810E94C80B0895EA
:101A7000E8E1F2E0E80FF11D80810E94F50B089586
:101A8000CF93DF93C8E1D2E089910E940D0C82E0F0
:101A9000C532D807C9F7DF91CF9108950E94400D54
:101AA00084E00E940D0C83E00E940D0C88E00E94EF
:101AB0000D0C81E00E940D0C82E00E940D0C089537
:101AC000F8941798E7E7F3E080818EBD0DB407FE28
:101AD000FDCF319683E0EC37F807B1F7179A789489
:101AE0000895E7E7F3E0ACE7B3E080819D91892BAF
:101AF000819383E0EC37F807C1F70895E7E7F3E057
:101B0000ACE7B3E09D91909580818923819383E038
:101B1000EC37F807B9F70895E7E7F3E0ACE7B3E08F
:101B200020819C91892F822319F090959223908394
:101B30001D92319683E0EC37F80791F708951F93D3
:101B4000182F84E00E940D0C123021F483E00E94D3
:101B5000C80B0FC083E00E940D0C83E00E94DE0BD7
:101B6000113011F483E003C01F3F19F484E00E9498
:101B7000B20B1F9108950F931F93CF93DF93182FEC
:101B800087FF04C086E10E94870C03C086E10E94A3
:101B90009B0C812F829586958695837080FF04C06B
:101BA00085E10E94870C03C085E10E949B0C1F7396
:101BB00039F0173110F48FEF11C0143218F41C50A3
:101BC00080E00CC0103318F4185181E007C01C33BA
:101BD00018F4145282E002C0105383E00E949F0D5B
:101BE000112331F40E94400D84E10E94870C1AC039
:101BF00084E10E949B0CCBE0D0E0012F10E0C017E5
:101C0000D10731F0FE01E35FFD4F80810E940D0C92
:101C10002196C831D10599F7035F1D4FF8018081E6
:101C20000E94B20BDF91CF911F910F910895AC01EB
:101C300020E0E0E009C0A40FB51F8C91E827F0E098
:101C4000EA5AFD4FE0812F5FA22FB0E0A617B70739
:101C500090F38E2F08950E94E50A8091C1038E3083
:101C6000D1F30E94380C0E94600D0895EF92FF920C
:101C70000F931F93CF93DF937C018B01C0E0D0E0E3
:101C800007C0F701EC0FFD1F80810E9444012196DF
:101C9000C017D107B0F3DF91CF911F910F91FF9043
:101CA000EF90089522E42093CC031092CD0322E01C
:101CB0002093CE039093CF038093D003ACECB3E09A
:101CC000E0E08D91E827F0E0EA5AFD4FE08183E003
:101CD000A13DB807B1F7EC93CD01059766E070E040
:101CE0000E94360E089590E89093CC031092CD0395
:101CF00091E09093CE038093CF03ACECB3E0E0E0AF
:101D00008D91E827F0E0EA5AFD4FE08183E0A03DA5
:101D1000B807B1F7EC93CD01049765E070E00E943D
:101D2000360E08951F920F920FB60F920BB60F92B8
:101D300011240F931F932F933F934F935F936F93B0
:101D40007F938F939F93AF93BF93CF93DF93EF9343
:101D5000FF931091CE0080915502882309F4FBC0B7
:101D60008091830390918403895E934030F00E94B8
:101D70004D0C0E94600D109281038091810380348C
:101D800048F4E82FF0E0E45FFB4F10838F5F80930F
:101D9000810304C00E94730E109281031092840389
:101DA0001092830320918103233008F4D4C0609102
:101DB0000C0490910D0480E070910E04E72FF0E088
:101DC000E82BF92B30E0CF0104962817390708F4E7
:101DD000C2C0AF014D5F5F4FFA01E45FFB4F9081DE
:101DE000E0E020E009C0A45FBB4F8C91E827F0E061
:101DF000EA5AFD4FE0812F5FA22FB0E0A417B5078C
:101E000090F39E17D9F0E0E020E009C0A45FBB4F3B
:101E10008C91E827F0E0EA5AFD4FE0812F5FA22F76
:101E2000B0E0A417B50790F38E2F90E00E94230135
:101E30001092810380E00E94730E8DC0613119F110
:101E4000623138F4613009F47FC0603109F07EC03E
:101E50005AC0603421F0613409F078C007C0809125
:101E60009203909193030E94520E73C0723009F056
:101E70006DC090910F0480E020911004820F911D9D
:101E80000E94B00166C0723009F060C080910F04FA
:101E9000C82FD0E033E0CC0FDD1F3A95E1F78091F9
:101EA0001004C80FD11D24E0CC0FDD1F2A95E1F7E7
:101EB00089E18093CC031092CD0380E18093CE031F
:101EC0000FEC13E0CE010E94E210F80181938F0124
:101ED0002196F3E00F3D1F07A9F7D8015397E0E0E3
:101EE0008D91E827F0E0EA5AFD4FE08123E0AF3D15
:101EF000B207B1F7E093DF03CD01439764E170E0EF
:101F00000E94360E26C0723109F580910F04C82F49
:101F1000D0E093E0CC0FDD1F9A95E1F7809110049B
:101F2000C80FD11D84E0CC0FDD1F8A95E1F701E1D8
:101F300014E0F80181918F01BE010E949E1021964C
:101F4000F4E001321F07A9F781E001C080E00E94A0
:101F5000730E10928103FF91EF91DF91CF91BF91AA
:101F6000AF919F918F917F916F915F914F913F9131
:101F70002F911F910F910F900BBE0F900FBE0F90DE
:101F80001F9018952C98803408F08FE3611160E45D
:101F9000442311F090E001C090E8882331F0682BD1
:101FA000962B98B92C9A2D9A0895962B98B9089546
:101FB000882311F0469A01C02D982C9808959F927D
:101FC000AF92BF92CF92DF92EF92FF920F931F9347
:101FD000CF93DF930E9491020E944D0C0E94E50A6C
:101FE0000E94E00A00E010E0CC24AA240E94E50A46
:101FF0008091C103843071F00E94D508DF91CF91A8
:102000001F910F91FF90EF90DF90CF90BF90AF9016
:102010009F90089580919A030E946F0C882331F459
:102020000E944D0C80919A030E945B0C0E94E00A72
:10203000882341F06091C80360939A0384E090E0A4
:102040000E946801802F0E949F0DC801880F991F70
:10205000800F911FE82EEE0CEE0CBC2CB294BB0C42
:10206000BB0C80ECB82287E1E80EC0E0D0E09E2CEB
:10207000FC2EFE01EA5AFC4FD0808D2D0E945D0A95
:10208000882381F08E2D8C0F6A2D4C2D0E94C20F5B
:10209000892D8C0F8B290E9427088C2F0E941A0DE6
:1020A000AA24A3948D2D0E94730A882341F08E2DBB
:1020B0008F0D8B290E945E088F2D0E94240D219682
:1020C000CD30D105A9F68FE00E945D0A882331F05A
:1020D0000230110574F40F5F1F4F0BC08EE00E9499
:1020E0005D0A882331F08FEF0F3F180711F0015080
:1020F000104085E10E945D0A882371F080E0CC20C9
:1021000009F481E0C82E882321F081E00E94B20BFF
:1021100003C081E00E940D0C86B190E08F73907037
:10212000892B09F463CF0E94890A882309F45ECFC2
:1021300080E00E94D80F0E94400D57CF282FF894BE
:1021400095E0289800000000000000009EBD0DB43E
:1021500007FEFDCF00000000000000001EBC0DB413
:1021600007FEFDCF8EB5289A000000000000000099
:1021700080FDE7CF28980000000086E08EBD0DB4FA
:1021800007FEFDCF00000000289A000000000000BC
:10219000000028980000000082E08EBD0DB407FE0C
:1021A000FDCF7EBD0DB407FEFDCF6EBD0DB407FEA5
:1021B000FDCF2EBD0DB407FEFDCF00000000289A14
:1021C00078940895282FF89428980000000083E060
:1021D0008EBD0DB407FEFDCF9EBD0DB407FEFDCF35
:1021E0002EBD0DB407FEFDCF000000001EBC0DB4D7
:1021F00007FEFDCF8EB5289A78940895892F8F71A8
:1022000084FD806E0895EF92FF920F931F93CF93FA
:10221000DF93C82FD0E023E0CC0FDD1F2A95E1F734
:10222000C60FD11DC05CDF4F95E0CC0FDD1F9A9526
:10223000E1F7EE24FF248701000F111F045B1B4F01
:10224000F80180819181892FBE010E949E10F801C2
:10225000808191812196BE010E949E100894E11C0C
:10226000F11C2196F0E1EF16F10429F7DF91CF91EF
:102270001F910F91FF90EF900895AF92BF92CF9270
:10228000DF92EF92FF920F931F93CF93DF93C82FAC
:10229000D0E053E0CC0FDD1F5A95E1F7C60FD11DFA
:1022A000C05CDF4F45E0CC0FDD1F4A95E1F7AA2463
:1022B000BB24CE010E94E210D82ECC247501EE0C76
:1022C000FF1C8CE494E0E80EF91EF701D182C08275
:1022D00000811181CE0101960E94E21090E0082B4E
:1022E000192BF701118300830894A11CB11C2296BD
:1022F000F0E1AF16B104E9F6DF91CF911F910F9194
:10230000FF90EF90DF90CF90BF90AF900895109224
:1023100070041092770410926C0480E00E94D80F31
:102320000E94380C0E948C0D0E94E00A0895809152
:102330006E0490916F04682F6770A3E0969587955F
:10234000AA95E1F78F700E94D41560916E04709188
:102350006F049B0140E050E0DA01C9018070907881
:10236000A070B070892F9A2FAB2FBB2780938B035F
:10237000DA01C90180709074A070B070892F9A2F13
:10238000AB2FBB2780938903207030724070507050
:10239000232F342F452F552720938A03109274043E
:1023A000872F8F7184FD806E089581E08093700483
:1023B00081E20E94B20B109289038091890380937D
:1023C0008A0380918A0380938B0310926C0410928D
:1023D000770480914C0490914D0490936F04809306
:1023E0006E048F5F9F4F89F01092730410927404F3
:1023F000109291030E949711809385038091650349
:1024000080FDFCCF81E080936C040E944D0C089508
:1024100081E08093710484E20E94B20B0E944D0C13
:1024200008951092710484E20E940D0C0E94380CF1
:102430000E948C0D1092770480E00E94D80F0895BE
:1024400080918503882321F483E00E940D0C0CC049
:1024500087FF07C083E00E940D0C84E00E94B20B4E
:10246000089583E00E94B20B84E00E940D0C089551
:10247000AF92BF92CF92DF92EF92FF921F93CF93D2
:10248000DF930E9494008091C803877080936D044D
:1024900010927204109271041092700410926C04E5
:1024A00010927704109273048FEF9FEF90936F0454
:1024B00080936E04109264030E944D0C0E948C0D58
:1024C000EE24EA94FE2CC12CA0E2DA2EA12CF0E43A
:1024D000BF2E0E94E50A8091C1038130B9F00E94AD
:1024E00091021092770410926C0480E00E94D80F41
:1024F0000E94380C0E94600DDF91CF911F91FF90D8
:10250000EF90DF90CF90BF90AF90089580917104CD
:10251000882359F580917004882339F50E94E00AD8
:10252000882359F08091C803877080936D0460916F
:1025300072040E943D110E944D0C80916D040E9416
:102540005B0C0E94B00A182F882351F00E94400DA6
:10255000612F61506093720480916D040E943D115F
:10256000809172048F5F0E94B30C81E00E945D0A2B
:10257000882379F080917004882319F00E948711D4
:1025800008C080917104882311F00E9411120E94EA
:10259000D51180917004882329F4809171048823D7
:1025A00009F451C0809173040E947B0C882311F4BC
:1025B0000E948C0D809173040E94650C80916E04C2
:1025C00090916F048F5F9F4F21F40E944E0D80E029
:1025D00034C080E00E940D0C80916E0490916F04D5
:1025E000E3E096958795EA95E1F78F700E945B0C82
:1025F00080916E0490916F0497FF04C088E00E9460
:10260000B20B03C088E00E940D0C80916E04909183
:102610006F04A0E0B0E096FF04C081E00E94B20B1E
:1026200003C081E00E940D0C80916E0490916F04B4
:10263000A0E0B0E095FF04C082E00E94B20B03C0AE
:1026400082E00E940D0C88E00E945D0A882331F42C
:1026500083E00E945D0A882309F470C080917004B1
:10266000882309F06BC00E94D80F809171048823E1
:1026700009F43CC088E00E945D0A8823A9F080919B
:10268000730490E00F97CCF5E0917304F0E0EE0F47
:10269000FF1FE45BFB4F808191818F5F9F4F69F14A
:1026A000809173048F5F1FC080917304882331F081
:1026B00017C0809173048F5F8093730480917304BB
:1026C00090E00F97E4F4E0917304F0E0EE0FFF1F49
:1026D000E45BFB4F808191818F5F9F4F51F70FC06B
:1026E0008091730481508093730409C088E00E9434
:1026F0005D0A882321F00E94081210927304E09171
:102700007304F0E0EE0FFF1FE45BFB4F80819181CB
:1027100090936F0480936E04109277048F5F9F4FA5
:1027200069F00E9497118093850310927404809140
:10273000650380FDFCCF81E08093770487E10E94F0
:102740005D0A882309F1809171048823B9F0809192
:10275000730490E00F974CF4E0917304F0E0EE0FF7
:10276000FF1FE25BFB4FF182E082F0926F04E09288
:102770006E040E94111280E00E940D0C80916D0485
:10278000609172040E94031180917104882309F4FE
:1027900070C180916E0490916F048F5F9F4F09F418
:1027A00002C184E10E945D0A8823F9F0E09173047C
:1027B000F0E0EE0FFF1FE45BFB4F808191818050C2
:1027C0009048918380838081918190936F0480935E
:1027D0006E04A0E0B0E080709078A070B070892F97
:1027E0009A2FAB2FBB2780938B0385E10E945D0A54
:1027F0008823F9F0E0917304F0E0EE0FFF1FE45B33
:10280000FB4F808191818A259B25918380838081E4
:10281000918190936F0480936E04A0E0B0E080708B
:102820009074A070B070892F9A2FAB2FBB27809324
:10283000890386E10E945D0A8823F9F0E091730420
:10284000F0E0EE0FFF1FE45BFB4F808191818C2550
:102850009D25918380838081918190936F048093E3
:102860006E04A0E0B0E080709072A070B070892F0C
:102870009A2FAB2FBB2780938A038FE00E94470AD1
:10288000882331F48EE00E94470A882309F479C036
:102890000E949B0AC82FDD27C7FDD0958FE00E94BC
:1028A0005D0A882329F48EE00E945D0A882351F096
:1028B0000E948C0D0E94400D83E00E940D0C84E06C
:1028C0000E940D0C8FE00E94470A882339F183E0B3
:1028D0000E94B20B8FEFCF3FD807C1F00E948C0D42
:1028E0003C2F222780916E0490916F04907E282BBC
:1028F000392B30936F0420936E04E0917304F0E061
:10290000EE0FFF1FE45BFB4F3183208380916F0448
:102910008F7184FD806E8093850330C08EE00E94AD
:10292000470A882309F43FC084E00E94B20B2FEFCE
:10293000CF3FD207D9F00E948C0D2C97CF71D07069
:102940003C2F222780916E0490916F04907E282B5B
:10295000392B30936F0420936E04E0917304F0E000
:10296000EE0FFF1FE45BFB4F3183208380916F04E8
:102970008F7184FD806E80938503845F0E942E0D8D
:1029800012C08FE00E94730A882329F48EE00E940F
:10299000730A882341F083E00E940D0C84E00E94BA
:1029A0000D0C0E948C0D8FE00E94470A882309F0CD
:1029B00060C08EE00E94470A882309F05AC00E9436
:1029C000C80A182F882329F40E94E00A882309F4F2
:1029D00045C00E940C0D0E944D0C112359F48091AA
:1029E0006E0490916F042FEF8F3F920721F0182F04
:1029F000177001C011501092770480E00E94D80F28
:102A0000412F50E08091C803282F30E093E0220F3F
:102A1000331F9A95E1F7422B532B50936F04409349
:102A20006E04E0917304F0E0EE0FFF1FE45BFB4FD8
:102A300051834083612F0E94D41510927404109228
:102A40008A0380918A03809389038091890380930C
:102A50008B031092850381E0809377040E942012FB
:102A600080916E0490916F048770907001960E941F
:102A7000BE0C80917004882309F42BCD0E94201293
:102A800080916E0490916F048770907001960E94FF
:102A9000BE0C1FCD1092710484E20E940D0C1092A6
:102AA000870380E00E940D0C0E948C0D0E94A50CF3
:102AB0000E944D0C8091C8030E945B0C80E00E9434
:102AC000D80F089581E08093710484E20E94B20BD4
:102AD0000E944D0C80E00E945B0C80E00E94D80FA9
:102AE0000895109277040E94A50C0E944D0C0E943C
:102AF0008C0D8091C8030E945B0C1092750481E2DA
:102B00000E940D0C80E00E94D80F1092CA048CEF36
:102B10000E94860808951092740481E080937504E1
:102B200081E20E94B20B80E00E94D80F8091640382
:102B3000882321F48091650380FDFCCF81E08093A0
:102B400077048093CA048AEF0E94860808950F9341
:102B50001F93CF93DF93182F062F0E94600DC12F74
:102B6000D0E093E0CC0FDD1F9A95E1F7C00FD11DA7
:102B700084E0CC0FDD1F8A95E1F700E010E0F8015A
:102B8000E758FB4F8081B8016C0F7D1F0E949E109B
:102B90000F5F1F4F0031110591F70E94600DDF910B
:102BA000CF911F910F9108950F931F93CF93DF93B0
:102BB000182F062F0E94600DC12FD0E033E0CC0FFC
:102BC000DD1F3A95E1F7C00FD11D24E0CC0FDD1FCA
:102BD0002A95E1F700E010E0C8018C0F9D1F0E94CC
:102BE000E210F801E758FB4F80830F5F1F4F003161
:102BF000110591F71092870380E00E94DE0B0E947E
:102C0000600DDF91CF911F910F9108959F92AF9228
:102C1000BF92CF92DF92EF92FF920F931F93CF93C9
:102C2000DF93B090C1031092760410927104109259
:102C3000750410927704109274041092910380919D
:102C40006403882319F40E94940004C00E94910236
:102C50000E94D8090E94E50A8091C80380937804F5
:102C6000609176040E94D4150E94380C8091C803AC
:102C70000E945B0CCC24C394AA24AA9440E4942E12
:102C80000E94E50A8091C1038B15D9F00E94910240
:102C90001092770480E00E94D80F0E94AE090E9433
:102CA000EC080E94380C0E94600DDF91CF911F91BB
:102CB0000F91FF90EF90DF90CF90BF90AF909F90DB
:102CC0000895909178048091C8039817D1F080916D
:102CD0007504882311F00E94711580917104882376
:102CE00011F00E944A158091C80380937804609186
:102CF00076040E94D4150E944D0C8091C8030E9456
:102D00005B0C809175048823D9F480917104882329
:102D1000B9F4809176048F5F0E94B30C0E94B00AD0
:102D2000182F882369F00E94400D812F0E94B30C58
:102D3000612F615060937604809178040E94D415CD
:102D400080E00E945D0A8823B1F080917504882399
:102D500091F082E20E94B20BC0E0D0E00E949E009F
:102D6000FE01E758FB4F80832196C031D105B1F7B2
:102D7000C09287030CC080E00E94730A882339F058
:102D800080917504882319F082E20E940D0C8091D5
:102D9000CA048823B9F080916403823099F4809149
:102DA000690390916A031816190664F48091690307
:102DB00090916A03039790936A03809369030E943A
:102DC000F4035ECF80916403823041F40E94B50821
:102DD000D82E882319F090E00E9423018091750479
:102DE000882399F080916403882329F481E00E946C
:102DF0005D0A882339F480916403823031F48CEFCA
:102E0000D81619F40E94711519C0809164038823A3
:102E100029F481E00E945D0A882341F480916403D3
:102E2000823061F48D2D8A5F823040F4809171048C
:102E3000882311F00E944A150E948B158091750419
:102E4000882329F480917104882309F439C1809181
:102E50007404E82EFF24E701C758DB4F18811F7365
:102E600085E10E945D0A882339F01F3329F08881AB
:102E700089258883C092870386E10E945D0A8823A2
:102E800059F01F33E9F0F701E758FB4F8081805874
:102E90008083C092870302C01F3391F0112381F019
:102EA000173110F40FEF0DC0143250F0103310F43E
:102EB00001E007C01C3310F003E003C002E001C0D2
:102EC00000E084E10E945D0A811110E08FE00E9421
:102ED0005D0A882339F01F3329F0112319F00230DD
:102EE0000CF4145F8EE00E945D0A882339F01F33D2
:102EF00029F0112319F00F3F09F01C5084E00E94C3
:102F00005D0A882331F08CE00802C0011124182FDB
:102F1000195E89E00E945D0A882331F08CE0080286
:102F2000C0011124182F185E85E00E945D0A8823D5
:102F300031F08CE00802C0011124182F175E8AE0DE
:102F40000E945D0A882331F08CE00802C001112440
:102F5000182F165E033009F463C086E00E945D0AF4
:102F6000882331F08CE00802C0011124182F155E6F
:102F700087E00E945D0A882331F08CE00802C001DE
:102F80001124182F145E8BE00E945D0A882331F013
:102F90008CE00802C0011124182F135E81E10E9409
:102FA0005D0A882331F08CE00802C0011124182F3B
:102FB000125E8CE00E945D0A882331F08CE00802EA
:102FC000C0011124182F115E82E10E945D0A88233E
:102FD00031F08CE00802C0011124182F105E8DE042
:102FE0000E945D0A882331F08CE00802C0011124A0
:102FF000182F1F5D80E10E945D0A882331F08CE06C
:103000000802C0011124182F1E5D83E10E945D0A91
:10301000882331F08CE00802C0011124182F1D5DB7
:10302000F701E758FB4F80818F3F11F41F3331F4D4
:10303000F701E758FB4F8081807C182BF701E75898
:10304000FB4F8081181701F180917104882331F0C2
:1030500080E00E94D80F81E00E94AE07E9E7F4E02B
:10306000EE0EFF1EF7011083C0928703809171045A
:10307000882351F0412F4295469546954170812F06
:103080008F7360E00E94C20F1F3F79F0812F0E9472
:10309000BB0D80918703882321F080E00E94C80B3C
:1030A0000FC080E00E940D0C0BC00E944E0D80E00E
:1030B0000E94DE0B83E00E94DE0B80E00E94B20BD8
:1030C00088E00E945D0A882331F483E00E945D0A53
:1030D000882309F49BC06091910380917104882337
:1030E00009F470C0162F111F1127111F812F0E9484
:1030F000D80F81E00E94AE0788E00E945D0A882315
:10310000A1F08091740490E00F9744F4E09174046E
:10311000F0E0E758FB4F80818F3F19F41092740460
:1031200020C0809174048F5F1AC08091740488233A
:1031300031F012C0809174048F5F80937404809189
:1031400074048F3070F4E0917404F0E0E758FB4FA2
:1031500080818F3F79F705C08091740481508093FE
:1031600074040E944D0C809174040E945B0CE091E9
:103170007404F0E0E758FB4F8081809391038F3F08
:1031800069F481E00E940D0C82E00E940D0C80E049
:103190000E94B20B80E00E94DE0B38C080E00E94EB
:1031A0000D0C80918703882319F080E00E94C80BE2
:1031B00080919103482F42954695469541708F73B3
:1031C000612F1EC088E00E945D0A8823F9F080917B
:1031D00075048823D9F40E94621510927404E0915A
:1031E0007404F0E0E758FB4F8081809391038F3F98
:1031F00069F0482F42954695469541708F7360E07F
:103200000E94C20F809191030E94BB0D87E10E9432
:103210005D0A882309F434CD80917104882369F014
:103220008091740490E00F9734F4E0917404F0E01E
:10323000E658FB4FA0820E944A158091C803609116
:1032400076040E94A7151092870380E00E94DE0B8F
:1032500017CDAC0120E030E0DA01A20FB31F8C9152
:10326000FB01E20FF31F9081891711F080E00895B0
:103270008C918F3F29F02F5F3F4F2032310561F74E
:1032800081E00895CF92DF92EF92FF920F931F9308
:10329000CF93DF93E090C10380916403882319F4F6
:1032A0000E94940002C00E949102809164038130C8
:1032B00019F40E94DF0902C00E94D8090E94380C4C
:1032C0000E948C0D1092A9048091A9048093890416
:1032D0008FEF8093AA048091AA0480938A0481E0EE
:1032E0000E94B30C1092CA041092730410927404DA
:1032F00010926F0410926E041092C904109286030B
:10330000109285030E944D0C8091C1038F3021F0F3
:103310008B3011F0873019F48091C80303C080917D
:10332000C803877080938C0380938D038091C803BA
:103330000E945B0CFF24DD24DA94CC24C3940E9409
:10334000E50A8091C1038E15F9F01092CA040E941B
:10335000AE090E94EC081092860310928503109229
:103360008A0310928B03109289030E94380C0E94EA
:103370008C0D0E94600DDF91CF911F910F91FF90F6
:10338000EF90DF90CF90089587E10E945D0A882337
:1033900021F180918E0390918F0386509D40C8F457
:1033A00080918E0390918F038E54914090F06091A4
:1033B0008E0370918F0380E69AEE0E94BF1C70937B
:1033C0008F0360938E0380918E0390918F030E94F0
:1033D000B00110928F0310928E0380E00E945D0A6C
:1033E000882349F00E94400D0E948C0D82E20E94C9
:1033F000B20B1092880380E00E94730A882379F14F
:1034000020E030E0F901E553FB4F8081F901E757F7
:10341000FB4F80832F5F3F4F2032310599F780911A
:10342000CA048823C9F420E030E0F901E757FB4FD4
:103430008081F901E755FB4F80832F5F3F4F20329A
:10344000310599F7809186038093850383E00E947C
:103450000D0C84E00E940D0C82E20E940D0C80E0B5
:103460000E94470A882351F110E00BC0E12FF0E0E1
:10347000E553FB4F8081883040F48F5F0E94B30C8E
:103480001F5F80918803181788F30E94C80A882359
:1034900009F43FC190918803903208F03AC1E92FB6
:1034A000F0E0E553FB4F81508083E92FEF5FE0931D
:1034B0008803F0E0E553FB4FD0822BC18FE00E94E0
:1034C000470A882331F48EE00E94470A882309F4D2
:1034D0006DC00E949B0A182F8FE00E945D0A88230E
:1034E00029F48EE00E945D0A882339F00E94400D85
:1034F0000E948C0D82E20E940D0C8FE00E94470A10
:10350000882301F184E00E940D0C83E00E94B20B3D
:103510001F3F11F0109386038091850387FD0AC039
:103520000E94380D882331F40E948C0D8091850310
:103530000E942E0D9091860380918503981761F16A
:10354000892F28C08EE00E94470A882329F183E052
:103550000E940D0C84E00E94B20B1F3F19F01C501A
:103560001093860380918503181664F0845F0E948F
:10357000380D882339F40E948C0D80918503845F77
:103580000E942E0D9091860380918503981721F05B
:10359000892F845F0E941A0D8091CA04882309F044
:1035A000B8C08091860380938503B3C08FE00E94EA
:1035B000730A882329F48EE00E94730A882321F07D
:1035C0000E94400D0E948C0D0E94B00A182F882383
:1035D00009F0C0C10E94E00A8823B9F18091C103BB
:1035E0008F3089F414C020E030E0F901E757FB4F39
:1035F0008081F901E755FB4F80832F5F3F4F2032D9
:10360000310599F714C08B3011F0873019F480918F
:10361000C80303C08091C803877080938D03809195
:10362000CA04882321F480918D0380938C038091B8
:10363000CA04882351F40E944D0C80918D030E948E
:103640005B0C809186038093850389E894E069EAA6
:1036500074E00E9429198823F9F480918A048F3F2D
:1036600049F48091AA048F3F29F48091A9048F5FC7
:103670000E94E70CC0E0D0E0FE01E757FB4F8081DD
:10368000893008F044C080818F5F0E94B30C21967E
:10369000C032D10589F73BC000E010E0E801C75512
:1036A000DB4F8881893098F58091CA048823C1F066
:1036B0008881E091C904F0E0E755FB4F90818917BC
:1036C00079F488818F5F0E94F20C8823D9F4888175
:1036D0008F5F0E94DC0C88818F5F0E94E70C12C014
:1036E000F801E755FB4F80818F5F0E94F20C882321
:1036F00011F00E948C0DF801E755FB4F80818F5F20
:103700000E94B30C0F5F1F4F0032110539F60E9463
:1037100020128091CA04882351F180916403823081
:1037200089F48091690390916A0318161906FCF4D4
:103730008091690390916A03039790936A03809341
:10374000690312C0813099F480916E0390916F03E8
:103750001816190664F480916E0390916F03039715
:1037600090936F0380936E030E94F403E8CD8091E1
:103770006403823019F40E94B508F82E8091640326
:10378000882349F481E00E945D0A882321F080911A
:10379000CA04882371F480916403823021F48CEF91
:1037A000F81661F506C0813049F50E94C6098823E4
:1037B00029F11092CA0480E00E94D80F0E94EC0800
:1037C00080916403813011F00E94AE0981E20E9471
:1037D0000D0C0E948C0D0E944D0C8091C1038F3006
:1037E00021F08B3011F0873019F48091C80303C0A9
:1037F0008091C80387700E945B0C68C0809164034D
:10380000882349F481E00E945D0A882321F0809199
:10381000CA04882391F080916403823031F48F2DA3
:103820008A5F823008F052C008C0813009F04EC073
:103830000E94B409882309F449C081E20E94B20BB6
:103840008091C1038F3021F08B3011F0873039F433
:103850006091A9048091C8030E94D41511C06091A1
:10386000A9048091C80387700E943D1180914C0487
:1038700090914D0490936F0480936E040E94971171
:103880001092910380916403823019F42BEFF216A9
:1038900031F01092C90410927404109273041092C3
:1038A000650310926A031092690310926D031092DF
:1038B0006F0310926E03C092CA048AEF0E948608BA
:1038C00080916403813011F00E94E60986E10E9434
:1038D0005D0A882389F090E080918A03882309F4A7
:1038E00091E090938A03992321F082E00E94B20B29
:1038F00003C082E00E940D0C85E10E945D0A8823CE
:1039000089F090E080918903882309F491E09093F5
:103910008903992321F081E00E94B20B03C081E06A
:103920000E940D0C84E10E945D0A882309F407CDF2
:1039300090E080918B03882309F491E090938B03AE
:10394000992321F088E00E94B20BF9CC88E00E9414
:103950000D0CF5CC0E940C0D115010938904809130
:1039600089048093CB04D0928A0480918A04809346
:10397000CC048091CA04882309F435CE58CEAA1B02
:10398000BB1B51E107C0AA1FBB1FA617B70710F04A
:10399000A61BB70B881F991F5A95A9F7809590957C
:1039A000BC01CD010895A1E21A2EAA1BBB1BFD018B
:1039B0000DC0AA1FBB1FEE1FFF1FA217B307E4070E
:1039C000F50720F0A21BB30BE40BF50B661F771F66
:1039D000881F991F1A9469F7609570958095909546
:0E39E0009B01AC01BD01CF010895F894FFCF0B
:1039EE007F206404050607111210130409050A0648
:1039FE00070B110C120D1013201B191C1A180F0C8B
:103A0E000E0B0D0A0920191A180C0B0A0922212572
:103A1E002320191A18241B1C0F0E0D04030A0C0B5D
:103A2E00090801020026271D1E1F1012111314155E
:103A3E0016170506070100070E091C1B1215383F45
:103A4E00363124232A2D70777E796C6B6265484F50
:103A5E00464154535A5DE0E7EEE9FCFBF2F5D8DF40
:103A6E00D6D1C4C3CACD90979E998C8B8285A8AFB0
:103A7E00A6A1B4B3BABDC7C0C9CEDBDCD5D2FFF8A0
:103A8E00F1F6E3E4EDEAB7B0B9BEABACA5A28F8810
:103A9E00818693949D9A2720292E3B3C35321F1800
:103AAE00111603040D0A5750595E4B4C45426F6870
:103ABE00616673747D7A898E878095929B9CB1B670
:103ACE00BFB8ADAAA3A4F9FEF7F0E5E2EBECC1C6D0
:103ADE00CFC8DDDAD3D4696E676075727B7C5156C0
:103AEE005F584D4A4344191E171005020B0C212630
:103AFE002F283D3A33344E49404752555C5B767120
:103B0E00787F6A6D64633E39303722252C2B06018F
:103B1E00080F1A1D1413AEA9A0A7B2B5BCBB96917F
:103B2E00989F8A8D8483DED9D0D7C2C5CCCBE6E1EF
:103B3E00E8EFFAFDF4F30409050A06070B110C125F
:043B4E000D10130043
:00000001FF
